:100000000AC018951895189518951895189518956B
:100010001895189518958FE181BD87E181BD8FED09
:100020008DBFC0ECE8EB4E2EDD275D2EEEE7F0E055
:10003000A0E6B0E088278D933197E9F766248FEF2B
:1000400087BB8FEF81BB80E088BB80E082BB81E013
:100050008093600000916000053010F009F011C03D
:1000600086E98093650080E180936400ECE7F1E02D
:100070008E2E9F2E57D0A0E68C918F5F8C9309F027
:10008000E9CF81E08093600000916000033010F0C0
:1000900009F011C084E68093650080E180936400DC
:1000A000ECE9F1E08E2E9F2E3DD0A0E68C918F5F83
:1000B0008C9309F0E9CF81E08093600000916000AB
:1000C000013010F009F011C08AEF8093650080E1E3
:1000D00080936400ECEBF1E08E2E9F2E23D0A0E6FF
:1000E0008C918F5F8C9309F0E9CF81E08093600061
:1000F00000916000013010F009F011C084E6809397
:10010000650080E180936400ECEDF1E08E2E9F2E7F
:1001100009D0A0E68C918F5F8C9309F0E9CF93CF43
:10012000F894FFCF81E080936100409164000091DA
:100130006100041710F009F020C0E82DF92DA3E6A6
:10014000C8950C9231968E2E9F2EE82DF92DA2E6A1
:10015000C8950C9231968E2E9F2EA3E68C9182BB71
:10016000A2E68C9188BBA5E68C91992750D0A1E698
:100170008C918F5F8C9309F0D8CF08950000010017
:1001800002000400080010002000400000010002EE
:1001900000040008001000200040008000800040A3
:1001A00000200010000800040002000140002000B0
:1001B000100008000400020001000000010102021A
:1001C00004040808101020204040008040402020F7
:1001D000101008080404020201010000000140029E
:1001E000200410080810042002400180400220046E
:1001F0001008081004200240010000003197F1F7B8
:100200000895689462F80895E89462F80895EF9369
:10021000FF93EE27E82BE92B31F0E8EEF3E031977E
:0C022000F1F70197D1F7FF91EF910895DD
:00000001FF
